:100000000C942A000C94F00F18950000189500002D
:10001000189500001895000018950000189500002C
:10002000189500001895000018950000189500001C
:10003000189500001895000018950000189500000C
:1000400018950000189500001895000018950000FC
:10005000189500008FE58DBFC0EDE8EC4E2E88E0CE
:100060008EBFD6E0F3E05F2EA89584B7082E877F79
:1000700084BF88E1992781BD91BDEEEFF7E0A0E64E
:10008000B0E088278D933197E9F78BE089B980E05C
:1000900080BD88E18AB96624D39AD29AD198B89A59
:1000A000B99ABA9ABB9ABC9AA298A39AA49AA59A0A
:1000B000A69AA79A8B9885B78C7F826085BFB59AE0
:1000C000B69A9A9AC99A839A78947BB770647BBFE0
:1000D00000EE1DE420EE30E0A1EBB0E00D931D93A7
:1000E0002D933C93A1EBB0E00D911D912D913C918E
:1000F000ADEFB0E00D931D932D933C93ADEFB0E0C9
:100100000D911D912D913C91A1E0B1E00D931D93B6
:100110002D933C93A5EFB0E0E0E1FFE20E94C41212
:100120000E94BF0680E08093050100910501053023
:1001300018F011F00C94B400E4E9F0E2A5E0B1E0AD
:100140008C919927A5E0B1E0AD90BB24AFEBB0E076
:10015000AA0DBB1D0E94DD15A5E0B1E08C918F5F5B
:100160008C9310F40C9495005A924A92A1EBB0E053
:100170000D911D912D913C91D2010D931D932D93C5
:100180003C9384E00E94AB140E94E00A229684E033
:100190000E9450105A924A92A1EBB0E00D911D912D
:1001A0002D913C91D2010D931D932D933C9384E0AE
:1001B0000E94AB140E94E00A229684E00E94501034
:1001C0000E943B01A1E0B1E04D915D916D917C9168
:1001D000ADEFB0E00D911D912D913C910E9428163C
:1001E00011F40C94F5000E94A803A5EBB0E04D912A
:1001F0005D916D917C91A1EBB0E00D911D912D91E0
:100200003C910E94281611F40C941C015A924A92B7
:10021000A1EBB0E00D911D912D913C91D2010D9378
:100220001D932D933C9384E00E94AB140E94E00A3E
:10023000229684E00E945010A1EBB0E00D911D9138
:100240002D913C91A5EBB0E00D931D932D933C9324
:10025000A7EAB0E04D915C91A5EAB0E00D911C9148
:100260000417150711F40C9437010E94DF040E9453
:100270004A060C94CA0081E00E94A51481E00E9405
:10028000A51482E00E94A51482E00E94A51482E0D9
:100290000E94A51400E513EC20E030E0A8E3B1E0F3
:1002A0000D931D932D933C930E942E17ECE4FFE2D7
:1002B0000E94BD10A0E6B0E036E20E9477100E94D6
:1002C0002B1781E0E0E6F0E002E00A93A0E9B0E05D
:1002D0000E94D116A0E6B0E00E941117EA2FFB2F72
:1002E00032970FEFA3E9B0E00E94D816A0E9B0E082
:1002F000E0E5FFE20E94171781E009F480E08F93A8
:10030000A3E9B0E0E4E5FFE20E94171781E009F4F9
:1003100080E09F91892B882311F40C94B10181E036
:10032000A885B9858C93A885B9850C91023018F001
:1003300011F00C94AD01DA9A84E690E00E942D1140
:10034000DA9884E690E00E942D11A885B9858C91F9
:100350008F5F8C9310F40C9493010C943B010C94DC
:10036000B201DA9A85E0E0E6F0E009E00A93A7E856
:10037000B0E00E94D116A7E8B0E00E949416A1EB6D
:10038000B0E00D931D932D933D93A1EBB0E00D9143
:100390001D912D913C91A3E1B1E00D931D932D93FF
:1003A0003C9340E054E465E978E0A1EBB0E00D91C6
:1003B0001D912D913C910E9428160CF402C00C94C2
:1003C000F601A1EBB0E00D911D912D913C9144E01F
:1003D00050E060E070E00E94AF14A1EBB0E00D933C
:1003E0001D932D933D93AC980C940902A1EBB0E0C2
:1003F0000D911D912D913C9140E058E468EE71E023
:100400000E942316A1EBB0E00D931D932D933D9315
:10041000AC9A82E1E0E6F0E006E00A93A5E9B0E0FC
:100420000E94D116A5E9B0E00E949416ADEAB0E0B2
:100430000D931D932D933D93ADEAB0E00D911D9169
:100440002D913C9144E050E060E070E00E94AF14D8
:10045000ADEAB0E00D931D932D933D9386E0E0E669
:10046000F0E003E00A93ACE9B0E00E94D116ACE9F9
:10047000B0E00E949416A5EAB0E00D931C938EE0C4
:10048000E0E6F0E004E00A93A0EAB0E00E94D116B2
:10049000A0EAB0E00E949416AE81BF810C93AE81B9
:1004A000BF810C91003011F00C94620201E010E069
:1004B00020E030E0ABE1B1E00D931D932D933C9330
:1004C0000C942003013011F00C9472020AE010E049
:1004D00020E030E0ABE1B1E00D931D932D933C9310
:1004E0000C9420030A3011F00C94820204E610E010
:1004F00020E030E0ABE1B1E00D931D932D933C93F0
:100500000C9420030B3011F00C94920208EE13E0CF
:1005100020E030E0ABE1B1E00D931D932D933C93CF
:100520000C9420030C3411F00C94A20208E213E2A4
:1005300020E030E0ABE1B1E00D931D932D933C93AF
:100540000C942003043611F00C94B20200E117E27F
:1005500020E030E0ABE1B1E00D931D932D933C938F
:100560000C942003053611F00C94C20200EA16E840
:1005700021E030E0ABE1B1E00D931D932D933C936E
:100580000C9420030E3611F00C94D20200E412E415
:100590002FE030E0ABE1B1E00D931D932D933C9340
:1005A0000C9420030F3611F00C94E20200E816E9D7
:1005B00028E930E0ABE1B1E00D931D932D933C931E
:1005C0000C942003083E11F00C94F20202E310E0B8
:1005D00020E030E0ABE1B1E00D931D932D933C930F
:1005E0000C942003093E11F00C9402030AEF10E072
:1005F00020E030E0ABE1B1E00D931D932D933C93EF
:100600000C942003023F11F00C94120304EF11E04C
:1006100020E030E0ABE1B1E00D931D932D933C93CE
:100620000C942003033F11F00C94200308E813E11D
:1006300020E030E0ABE1B1E00D931D932D933C93AE
:1006400088E1E0E6F0E001E00A93AB81BC810E9422
:10065000D116AA81BB810E949416ABEAB0E00C933C
:1006600089E1E0E6F0E001E00A93A981BA810E9405
:10067000D116A881B9810E949416ACEAB0E00C931F
:100680008DE1E0E6F0E001E00A93AD81BE810E94D9
:10069000D116AC81BD810E949416AAEAB0E00C93F9
:1006A000A3E3B0E00C9102FB81E00EF080E08F93B9
:1006B0000091A900013081E009F480E09F91892335
:1006C000882311F40C94740382E50E94C41088E519
:1006D0000E94C4108BE30E94C410DB98C49881E090
:1006E0008093A9000C949603A3E3B0E00C9102FB65
:1006F00081E00EF480E08F930091A900013081E049
:1007000009F080E09F918923882311F40C949603CB
:1007100084E50E94C41088E50E94C4108BE30E9407
:10072000C410DB9AC49A80E08093A9000091AA00CB
:10073000013011F00C94A003DB9AC49A0C94A2032C
:10074000DB98C49888E0481A80E0580A2A960895F1
:10075000ADEFB0E00D911D912D913C91A1E0B1E084
:100760004D915D916D917C910E942316AFE0B1E0B7
:100770000D931D932D933D93AFE0B1E00D911D912D
:100780002D913C9144E050E060E070E00E94AF1495
:10079000AFE0B1E00D931D932D933D93AFE0B1E039
:1007A0000D911D912D913C91ABE1B1E04D915D9189
:1007B0006D917C910E94AF14AFE0B1E00D931D9359
:1007C0002D933D93AC9B0C94F703AFE0B1E00D91FA
:1007D0001D912D913C9144E050E060E070E00E945A
:1007E000CB10AFE0B1E04D935D936D937D93A1EBA2
:1007F000B0E00D911D912D913C91AFE0B1E04D9194
:100800005D916D917C910E941E16A1EBB0E00D935D
:100810001D932D933D9340E452E46FE070E0A1EB13
:10082000B0E00D911D912D913C910E9428160CF481
:1008300002C00C94250400E412E42FE030E0A1EBA8
:10084000B0E00D931D932D933C9340E856E36EEB7F
:1008500076E2A1EBB0E00D911D912D913C910E94AB
:1008600028161CF011F00C9437040C94410400E895
:1008700015E528EC30E2A1EBB0E00D931D932D932C
:100880003C93ADEFB0E00D911D912D913C91A1E015
:10089000B1E00D931D932D933C935A924A92A1EB94
:1008A000B0E00D911D912D913C91D2010D931D93BE
:1008B0002D933C9384E00E94AB140E94E00A2296A0
:1008C00084E00E9450105A924A92A1EBB0E00D9140
:1008D0001D912D913C91D2010D931D932D933C932D
:1008E00084E00E94AB140E947A04229684E00E9465
:1008F000501008958CE00E94A5148EE00E94A5146B
:10090000AC9B0C949704AC81BD810D911D912D91F0
:100910003C9140E058E468EE71E00E941E16AC8104
:10092000BD810D931D932D933D930C94A904AC812F
:10093000BD810D911D912D913C9144E050E060E00E
:1009400070E00E94CB10AC81BD814D935D936D939F
:100950007D93AA81BB81EC81FD810E943E16EA81D4
:10096000FB81A0EBB3E00E94C616E0EBF3E0AA81A6
:10097000BB81112722270BE033270E94E015A881B5
:10098000B981E6E5FFE20E94D214EA81FB81A881E9
:10099000B9810E946E100E94C616A881B9810E947A
:1009A0006E10E4E5FFE20E94D214A881B9810E9492
:1009B000B7108AE1481A80E0580A24960895A5EAFB
:1009C000B0E00D911C910A3050E015070CF402C004
:1009D0000C94EE040C94DF040C944106A5EAB0E0FC
:1009E0000D911C91063252E015071CF011F00C9489
:1009F000FB040C94FF040C94DF040C944106A5EA5C
:100A0000B0E00D911C910A3050E0150780E00CF029
:100A100081E08F93A5EAB0E00D911C910E3150E07A
:100A2000150781E014F009F080E09F918923882365
:100A300011F40C941F0576E078BB0C944106A5EAEE
:100A4000B0E00D911C910E3150E0150780E00CF0E4
:100A500081E08F93A5EAB0E00D911C91023350E044
:100A6000150781E014F009F080E09F918923882325
:100A700011F40C943F0575E078BB0C944106A5EA8F
:100A8000B0E00D911C91023350E0150780E00CF0AE
:100A900081E08F93A5EAB0E00D911C91003550E004
:100AA000150781E014F009F080E09F9189238823E5
:100AB00011F40C945F0574E078BB0C944106A5EA30
:100AC000B0E00D911C91003550E0150780E00CF06E
:100AD00081E08F93A5EAB0E00D911C91083750E0BA
:100AE000150781E014F009F080E09F9189238823A5
:100AF00011F40C947F0573E078BB0C944106A5EAD1
:100B0000B0E00D911C91083750E0150780E00CF023
:100B100081E08F93A5EAB0E00D911C91003A50E07E
:100B2000150781E014F009F080E09F918923882364
:100B300011F40C949F0572E078BB0C944106A5EA71
:100B4000B0E00D911C91003A50E0150780E00CF0E8
:100B500081E08F93A5EAB0E00D911C910E3B50E02F
:100B6000150781E014F009F080E09F918923882324
:100B700011F40C94BF0571E078BB0C944106A5EA12
:100B8000B0E00D911C910E3B50E0150780E00CF099
:100B900081E08F93A5EAB0E00D911C910C3D50E0EF
:100BA000150781E014F009F080E09F9189238823E4
:100BB00011F40C94DF0570E078BB0C944106A5EAB3
:100BC000B0E00D911C910C3D50E0150780E00CF059
:100BD00081E08F93A5EAB0E00D911C910E3051E0B9
:100BE000150781E014F009F080E09F9189238823A4
:100BF00011F40C94FF0579E078BB0C944106A5EA4A
:100C0000B0E00D911C910E3051E0150780E00CF022
:100C100081E08F93A5EAB0E00D911C91003951E07D
:100C2000150781E014F009F080E09F918923882363
:100C300011F40C941F0678E078BB0C944106A5EAE9
:100C4000B0E00D911C91003951E0150780E00CF0E7
:100C500081E08F93A5EAB0E00D911C91063252E03D
:100C6000150781E014F009F080E09F918923882323
:100C700011F40C943F0677E078BB0C9441060C9479
:100C8000DF04A5EAB0E08D919C91A7EAB0E08D93D6
:100C90009C93089587E00E94A51485E00E94A51406
:100CA00081E00E94A514AFE1B1E08C918F5F8C933D
:100CB00000911F01043111F00C94B70680E080937D
:100CC0001F010E942E17EAE5FFE20E94BD10AC81D1
:100CD000BD8136E00E9477100E942B1781E0EC81E5
:100CE000FD8104E00A93AB81BC810E94D116AA81E8
:100CF000BB81E0E6FFE20E94171711F40C94840612
:100D00000C94B9060C94940685E0EC81FD8101E019
:100D10000A93AB81BC810E94D116AA81BB810E943B
:100D20009416A881B9810C93A881B9810C910130E6
:100D300011F00C949E06AF9A0C949F06AF98A88170
:100D4000B9810C91023011F00C94A906AE9A0C9462
:100D5000AA06AE98A881B9810C91033011F00C94C9
:100D6000B406AD9A0C94B506AD980C94B9060C94E3
:100D7000B9068DE0481A80E0580A2696089581E069
:100D80000E94A51481E00E94A51484E00E94A5148D
:100D9000AC81BD81BA93AA935A924A9287E8D20154
:100DA0008C9381E00E94AB140E94D10F249681E0C5
:100DB0000E945010AC81BD818C9181608C935A92BD
:100DC0004A9287E8D2018C9381E00E94AB145A9238
:100DD0004A92A885B9858C91D2018C9381E00E94BA
:100DE000AB140E94BF0F249682E00E94501081E055
:100DF000AC81BD818C93AC81BD810C91003011F42C
:100E00000C941B07AC81BD81BA93AA935A924A9263
:100E100087E8D2018C9381E00E94AB140E94D10F2D
:100E2000249681E00E945010AC81BD818C9181702C
:100E30008C930C94FB0681E08093050100910501E1
:100E4000063018F011F00C944D070091050146E0B2
:100E5000040FA6E0B1E00C93A5E0B1E0AD90BB2497
:100E6000A8EBB0E0AA0DBB1DBA93AA935A924A927E
:100E700080910601D2018C9381E00E94AB140E9404
:100E8000D10F249681E00E945010A5E0B1E08C9132
:100E90008F5F8C9310F40C941E07A9EBB0E00C91BB
:100EA00011272227332740EE50E060E070E00E94D7
:100EB0001F11A5ECB0E00D931D932D933D9395E08C
:100EC000A5ECB0E00E94F914A5ECB0E00D911D91E5
:100ED0002D913C9144E050E060E070E00E941E16CD
:100EE000A5ECB0E00D931D932D933D930091B900B7
:100EF0004FE10423AC81BD810C9392E0AC81BD81B4
:100F00000E94D8140091BA0040EC0423AA81BB814E
:100F10000C9396E0AA81BB810E94F114AC81BD8143
:100F20000C91112722273327AA81BB814C91552789
:100F3000662777270E941E16A9ECB0E00D931D933B
:100F40002D933D9340E050E060E070E0A9ECB0E00C
:100F50000D911D912D913C910E94281611F00C9439
:100F6000BD0701E010E020E030E0A9ECB0E00D9317
:100F70001D932D933C930C94DD070091C90041E033
:100F80000423AC81BD810C93AC81BD810C910030F8
:100F900011F40C94DD07A9ECB0E00D911D912D9199
:100FA0003C9141E050E060E070E00E941E16A9EC28
:100FB000B0E00D931D932D933D93AAEBB0E00C91FF
:100FC0001127222733274FE350E060E070E00E94B2
:100FD0001F11A881B9810D931D932D933D9394E02A
:100FE000A881B9810E94E0140091BB0040EF042366
:100FF000AC81BD810C9394E0AC81BD810E94F11461
:10100000A881B9810D911D912D913C91AC81BD813B
:101010004C915527662777270E941E16A881B98113
:101020000D931D932D933D93A881B981E7E0F1E0E5
:101030000E940E14ABEBB0E00C911127222733274E
:101040004FE050E060E070E00E941F11A881B9817C
:101050000D931D932D933D9398E0A881B9810E9433
:10106000E014A881B9810D911D912D913C91ACEBBB
:10107000B0E04C915527662777270E941E16A8815D
:10108000B9810D931D932D933D9398E0A881B9816B
:101090000E94E014A881B9810D911D912D913C9180
:1010A000ADEBB0E04C915527662777270E941E16BE
:1010B000A881B9810D931D932D933D9398E0A8814C
:1010C000B9810E94E014A881B9810D911D912D91E3
:1010D0003C91AEEBB0E04C915527662777270E94F4
:1010E0001E16A881B9810D931D932D933D93A88160
:1010F000B981E5EDF0E00E940E14A5EDB0E0BA93E1
:10110000AA93E8E1FFE2ADECB0E00E94C412E5ED85
:10111000F0E00E94FB112296A5EDB0E0BA93AA93ED
:10112000A5EDB0E0E7E0F1E00E9454112296A5ECB5
:10113000B0E0E7E0F1E00E940E14ADEDB0E0BA934C
:10114000AA93E0E2FFE2ADECB0E00E94C412EDEC45
:10115000F0E0A7E0B1E00E948F112296A9ECB0E088
:10116000E7E0F1E00E940E14ADEDB0E0BA93AA936F
:10117000A7E0B1E0EDEDF0E00E948F112296ADED19
:10118000B0E0BA93AA93A5EDB0E0EDEDF0E00E94D7
:10119000FB112296EDEDF0E0A5EEB0E00E94E31227
:1011A000ADEEB0E0E0E0F0E098E00E94FA16ADEEBF
:1011B000B0E0E8E2FFE20E949D1280E010F009F04A
:1011C00081E08F93ADEEB0E0E0E3FFE20E949D127C
:1011D00081E008F080E09F91892B882311F40C9422
:1011E000F908ADEDB0E0E8E3FFE20E94C4120C9410
:1011F000FF08EDEEF0E0ADEDB0E00E94E31286E016
:10120000481A80E0580A2696089584E00E94A514A2
:1012100084E00E94A51484E00E94A51484E00E944A
:10122000A5149AE0A885B9850E94F91405E51DE783
:1012300024E530E0A885B9854D915D916D917C9153
:101240000E94CB10AC81BD814D935D936D937D93D6
:1012500008E415E428E430E0A885B9854D915D9156
:101260006D917C910E94CB10AE81BF814D935D93B7
:101270006D937D9392E0AC81BD810E94F914AC81A5
:10128000BD810C9142E00E940117A6E0B1E08C9371
:1012900000910601013011F00C946009AC81BD8110
:1012A0000D911D912D913C9141E050E060E070E086
:1012B0000E941E16AC81BD810D931D932D933D930D
:1012C000AE81BF810D911D912D913C914BE050E07D
:1012D00060E070E00E94CB10AE81BF814D935D93C2
:1012E0006D937D93AE81BF810C9142E00E94011706
:1012F000A6E0B1E08C9300910601013011F00C944E
:101300009309AE81BF810D911D912D913C9141E0DA
:1013100050E060E070E00E942316AE81BF810D9323
:101320001D932D933D93AE81BF810D911D912D9104
:101330003C9141E050E060E070E00E941E16AE81FA
:10134000BF810D931D932D933D9340E850E060E0E5
:1013500070E0AC81BD810D911D912D913C910E9459
:1013600028161CF011F00C94B7090C94C10900E880
:1013700010E020E030E0AC81BD810D931D932D93F2
:101380003C9340E050E060E070E0AE81BF810D91A1
:101390001D912D913C910E9428161CF011F00C9487
:1013A000DB0901E010E020E030E0AE81BF810D9369
:1013B0001D932D933C9300E010E020E030E0A881E5
:1013C000B9810D931D932D933C9381E0809305018A
:1013D00000910501063018F011F00C94B60AA885AA
:1013E000B9850D911D912D913C91A5E0B1E0AD9095
:1013F000BB24AEEBB0E0AA0DBB1D4C915527662770
:1014000077270E94AF14AA81BB810D931D932D9362
:101410003D93AA81BB810D911D912D913C91AC8191
:10142000BD814D915D916D917C910E94AF14AA8117
:10143000BB810D931D932D933D9348E455E468E4DF
:1014400070E0AA81BB810D911D912D913C910E946C
:1014500028160CF002C00C94AE0A45E55DE764E581
:1014600070E0AA81BB810D911D912D913C910E944C
:1014700028161CF011F00C94AE0A40E050E060E039
:1014800070E0A881B9810D911D912D913C910E9430
:10149000281611F00C94740AAA81BB810D911D913C
:1014A0002D913C91A881B9810D931D932D933C936F
:1014B000A5E0B1E0AD90BB24AEEBB0E0AA0DBB1D42
:1014C0008C91A5ECB0E08D9388278D938D938C93B0
:1014D000AC81BD810D911D912D913C91A9ECB0E0A5
:1014E0000D931D932D933C93A881B9814D915D91EE
:1014F0006D917C91AA81BB810D911D912D913C91A3
:101500000E9428161CF011F00C94AE0AAA81BB812F
:101510000D911D912D913C91A881B9810D931D9341
:101520002D933C93A5E0B1E0AD90BB24AEEBB0E0D1
:10153000AA0DBB1D8C91A5ECB0E08D9388278D93EF
:101540008D938C93AC81BD810D911D912D913C911A
:10155000A9ECB0E00D931D932D933C93A5E0B1E071
:101560008C918F5F8C9310F40C94E809AC81BD8151
:101570000D911D912D913C9142E050E060E070E0B2
:101580000E942316AC81BD810D931D932D933D9335
:10159000AE81BF814D915D916D917C91AC81BD819A
:1015A0000D911D912D913C910E9428161CF011F077
:1015B0000C94E50980E1481A80E0580A28960895BD
:1015C00084E00E94A51484E00E94A51484E00E9497
:1015D000A51481E00E94A51481E00E94A51481E079
:1015E0000E94A51481E00E94A51481E00E94A51428
:1015F00088E00E94A51484E00E94A51484E00E9463
:10160000A5140091AA00003081E009F080E08F93DA
:101610000091AB00003081E009F080E09F918923C8
:101620008F930091AC00003081E009F080E09F9141
:101630008923882311F40C942F0BA1EBB0E00D91BA
:101640001D912D913C9140EA5CE860E070E00E94C1
:101650002316AE89BF890D931D932D933D93009161
:10166000AA00003081E009F080E08F930091AB0088
:10167000003081E009F080E09F9189238F930091F1
:10168000AC00013081E009F080E09F91892388233C
:1016900011F40C945D0BA1EBB0E00D911D912D9117
:1016A0003C9140EA5CE860E070E00E942316AE895D
:1016B000BF890D931D932D933D930091AA00003097
:1016C00081E009F080E08F930091AB00013081E070
:1016D00009F080E09F9189238F930091AC00013045
:1016E00081E009F080E09F918923882311F40C9414
:1016F0009F0BA1EBB0E00D911D912D913C9140EA23
:101700005CE860E070E00E942316AE89BF890D930B
:101710001D932D933D93AE89BF890D911D912D9100
:101720003C91ADEAB0E04D915D916D917C910E944C
:101730001E16AE89BF890D931D932D933D93009185
:10174000AA00003081E009F080E08F930091AB00A7
:10175000013081E009F080E09F9189238F9300910F
:10176000AC00003081E009F080E09F91892388235C
:1017700011F40C94E10BA1EBB0E00D911D912D91B2
:101780003C9140EA5CE860E070E00E942316AE897C
:10179000BF890D931D932D933D93AE89BF890D9104
:1017A0001D912D913C91ADEAB0E04D915D916D910F
:1017B0007C910E941E16AE89BF890D931D932D93B7
:1017C0003D930091AA00013081E009F080E08F9301
:1017D0000091AB00003081E009F080E09F91892307
:1017E0008F930091AC00003081E009F080E09F9180
:1017F0008923882311F40C94090CA1EBB0E00D911E
:101800001D912D913C91AE89BF890D931D932D9310
:101810003C930091AA00013081E009F080E08F93B1
:101820000091AB00013081E009F080E09F918923B5
:101830008F930091AC00003081E009F080E09F912F
:101840008923882311F40C94310CA1EBB0E00D91A5
:101850001D912D913C91AE89BF890D931D932D93C0
:101860003C930091AA00013081E009F080E08F9361
:101870000091AB00013081E009F080E09F91892365
:101880008F930091AC00013081E009F080E09F91DE
:101890008923882311F40C94610CA1EBB0E00D9125
:1018A0001D912D913C91ADEAB0E04D915D916D910E
:1018B0007C910E941E16AE89BF890D931D932D93B6
:1018C0003D930091AA00013081E009F080E08F9300
:1018D0000091AB00003081E009F080E09F91892306
:1018E0008F930091AC00013081E009F080E09F917E
:1018F0008923882311F40C94910CA1EBB0E00D9195
:101900001D912D913C91ADEAB0E04D915D916D91AD
:101910007C910E941E16AE89BF890D931D932D9355
:101920003D935A924A92A88DB98D0D911D912D919A
:101930003C91D2010D931D932D933C9384E00E9422
:10194000AB140E940509229684E00E945010A5EC79
:10195000B0E0E7E0F1E00E940E14AE89BF89EC81AF
:10196000FD810E940E14A5EDB0E0BA93AA93AE815A
:10197000BF81E7E0F1E00E948F112296A9ECB0E070
:10198000E7E0F1E00E940E14A5EDB0E0BA93AA934F
:10199000A7E0B1E0E5EDF0E00E948F112296C99931
:1019A0000C94FA0CA5EFB0E0BA93AA93E0E4FFE23E
:1019B000ADECB0E00E94C412E5EFF0E00E948F11A0
:1019C0002296ADEDB0E0BA93AA93A5EFB0E0EDEDAD
:1019D000F0E00E9454112296A5EFB0E0E0E1FFE2B2
:1019E0000E94C412E0E0F0E0ADEDB0E098E07BE7EB
:1019F0000E94E916A5EDB0E0BA93AA93ADEDB0E070
:101A0000E5EDF0E00E94FB11229681E08093050154
:101A100000910501063018F011F00C94210D80E0C2
:101A2000A5E0B1E0AD90BB24A8EBB0E0AA0DBB1DD2
:101A30008C93A5E0B1E08C918F5F8C9310F40C94A3
:101A4000080DA5ECB0E00D911D912D913C9144E065
:101A500050E060E070E00E942316A5ECB0E00D932A
:101A60001D932D933D9395E0A5ECB0E00E94E0140A
:101A70008091C5008093B90041E050E060E070E0E3
:101A8000A9ECB0E00D911D912D913C910E9428167A
:101A900011F00C94570D00E010E020E030E0A9ECCC
:101AA000B0E00D931D932D933C930C94770D009112
:101AB000C90041E00423AC85BD850C93AC85BD8590
:101AC0000C91003011F00C94770DA9ECB0E00D9161
:101AD0001D912D913C9141E050E060E070E00E944A
:101AE0002316A9ECB0E00D931D932D933D93009127
:101AF000B90040EE0423AA85BB850C938091C900F0
:101B0000A885B9858C9392E0A885B9850E94F114C7
:101B1000AA85BB850C91A885B9854C91042BA9EBAE
:101B2000B0E00C930091C90043E00423AE81BF8173
:101B30000C9396E0AE81BF810E94D814AE81BF8124
:101B40008C918093BA00E5EDF0E0A7E0B1E00E944F
:101B50004612AC81BD81BA93AA93A7E0B1E0E5ED4E
:101B6000F0E00E943F112296EC81FD81AA81BB81A9
:101B70000E942C1494E0AA81BB810E94F914AA81CE
:101B8000BB810C914FE30423AE85BF850C9300917C
:101B9000BA00AE85BF854C91042BAAEBB0E00C9344
:101BA000A7E0B1E0BA93AA93E8E1FFE2ADECB0E0C0
:101BB0000E94C412E7E0F1E00E948F112296E7E054
:101BC000F1E0A881B9810E942C14A881B9810D91FE
:101BD0001D912D913C91AC89BD890D931D932D9341
:101BE0003C9398E1AC89BD890E94F914AC89BD8908
:101BF0000C914FEF0423ABEBB0E00C93EC81FD8133
:101C0000AA81BB810E942C1494E0AA81BB810E940E
:101C1000E0140091BB00AA81BB814C91042BABEB7B
:101C2000B0E00C93A881B9810D911D912D913C914B
:101C3000AA89BB890D931D932D933C9390E1AA89AA
:101C4000BB890E94F914AA89BB890C914FEF042328
:101C5000ACEBB0E00C93A881B9810D911D912D9151
:101C60003C91A889B9890D931D932D933C9398E0DD
:101C7000A889B9890E94F914A889B9890C914FEFF4
:101C80000423ADEBB0E00C93A881B9810C914FEF28
:101C90000423AEEBB0E00C93AE85BF85BA93AA9354
:101CA0005A924A9289E8D2018C9381E00E94AB1447
:101CB0000E94D10F249681E00E945010AE85BF850E
:101CC0008C9180618C935A924A9289E8D2018C93CC
:101CD00081E00E94AB145A924A92AA89BB898C91E6
:101CE000D2018C9381E00E94AB140E94BF0F249616
:101CF00082E00E94501081E080930501009105016F
:101D0000063018F011F00C94B30E0091050146E076
:101D1000040FA6E0B1E00C935A924A92809106011A
:101D2000D2018C9381E00E94AB145A924A92A5E0B2
:101D3000B1E0AD90BB24A8EBB0E0AA0DBB1D8C9127
:101D4000D2018C9381E00E94AB140E94BF0F2496B5
:101D500082E00E945010A5E0B1E08C918F5F8C93DF
:101D600010F40C947E0EAE85BF85BA93AA935A9256
:101D70004A9289E8D2018C9381E00E94AB140E94C0
:101D8000D10F249681E00E945010AE85BF858C91C2
:101D90008F7E8C935A924A9289E8D2018C9381E08B
:101DA0000E94AB145A924A92AA89BB898C91D201A3
:101DB0008C9381E00E94AB140E94BF0F249682E0B6
:101DC0000E945010AE85BF85BA93AA935A924A9248
:101DD00087E8D2018C9381E00E94AB140E94D10F5E
:101DE000249681E00E945010AE85BF858C9180645E
:101DF0008C93A4E2B1E04D915D916D917C91A3E152
:101E0000B1E00D911D912D913C910E94281680E02A
:101E10000CF081E08F93A8E2B1E04D915D916D915E
:101E20007C91A3E1B1E00D911D912D913C910E9417
:101E3000281681E014F009F080E09F91892B882317
:101E400011F40C94B90FA3E1B1E00D911D912D9106
:101E50003C91A0E2B1E00D931D932D933C93E3E1FF
:101E6000F1E00E943E150E945D15ACE2B1E00E94D7
:101E70008115E8E4FFE20E94C815ECE2F1E00E945F
:101E80003E150E949315EDE0F0E0ACE2B1E00E9457
:101E9000CB16ECE2F1E00E940A15A0E3B1E0EDE020
:101EA000FF270E94CB16A0E2B1E00D911D912D916C
:101EB0003C91A0E3B1E04D915D916D917C910E94C8
:101EC0001E16A4E2B1E00D931D932D933D93A0E265
:101ED000B1E00D911D912D913C91A0E3B1E04D91A8
:101EE0005D916D917C910E942316A8E2B1E00D9363
:101EF0001D932D933D935A924A9287E8D2018C9379
:101F000081E00E94AB145A924A92AA89BB898C91B3
:101F1000D2018C9381E00E94AB140E94BF0F2496E3
:101F200082E00E94501081E0AE85BF858C93AE8523
:101F3000BF850C91003011F40C94B70FAE85BF85AE
:101F4000BA93AA935A924A9287E8D2018C9381E07D
:101F50000E94AB140E94D10F249681E00E94501081
:101F6000AE85BF858C9180748C930C94970F0C94E4
:101F7000B90F81E2481A80E0580A669608950E94D7
:101F800036171AEA0E944E17AA81BB811C910E9443
:101F90004E17A881B9811C910E944E170E944517C7
:101FA000089580E080933C010E9436171AEA0E944F
:101FB0004E17A881B9811C910E944E170E943617B6
:101FC0001BEA0E944E170E946B17ACE3B1E01C9312
:101FD0000E94451780913C01AA81BB818C93089592
:101FE0000F921F922F923F924F925F927F92AF92E9
:101FF000BF920F931F932F933F934F935F936F93D2
:102000007F938F939F93AF93BF93CF93DF93EF9380
:10201000FF938FB78F93C99B0C941D1083990C94D9
:102020001710ADEFB0E00E9454100C941B10ADEFF0
:10203000B0E00E9461100C942C1083990C9428102D
:10204000A5EFB0E0A5EFB0E00E947B120C942C103D
:10205000A5EFB0E00E947E1270E47ABF8F918FBF2F
:10206000FF91EF91DF91CF91BF91AF919F918F91B0
:102070007F916F915F914F913F912F911F910F91A0
:10208000BF90AF907F905F904F903F902F901F90A8
:102090000F90189504050607090B481A590A089568
:1020A000481A8827580A08950D911D912D913C9149
:1020B0000F5F1F4F2F4F3F4F3C932E931E930E9356
:1020C00008950D911D912D913C910150104020409B
:1020D00030403C932E931E930E9308958F938D91D1
:1020E0008823E9F711978F910895A0EBB3E01AD0F8
:1020F000803089F0883091F08D3039F03323B9F396
:102100008D933A9563FE40D0F2CF63FC04C08DE01E
:102110003BD08AE039D088278C93089535D0119729
:102120003395E5CF0F931F932F933F93AF93BF93B7
:10213000A8E3B1E00D911D912D913C915F990BC0E9
:102140008827802B812B822B832B39F00150104064
:1021500020403040F3CF8CB101C08827BF91AF91B0
:102160003F912F911F910F910895A0EBB3E08D91B6
:10217000882311F009D0FBCF08950E94C415802D4B
:1021800011F002D0FACF08955D9BFECF8CB908956F
:1021900000FC05D0089530D005D001F8F9CF37D034
:1021A0003FD00895842F952FA62FB72FE894452B65
:1021B000462B472B11F468940895402F512F622F1E
:1021C000732F0027112722273327F0E2440F551FD2
:1021D000661F771F001F111F221F331F081B190BBB
:1021E0002A0B3B0B416028F4080F191F2A1F3B1FC5
:1021F0004E7FFA9559F708950024E89477FF02C0BE
:1022000006D0689400F809D010F80124089512D07F
:102210004F5F5F4F6F4F7F4F0895E89437FF0895EA
:1022200000951095209530950F5F1F4F2F4F3F4F12
:10223000689408954095509560957095089504238D
:1022400015232623372308953197F1F708956894CD
:1022500062F80895E89462F80895EF93FF93EE27EB
:10226000E82BE92B31F0EDECFAE03197F1F701972B
:10227000D1F7FF91EF9108957CD204D09EC10F0158
:1022800001D09EC1FD01FF93EF9387818F9390E86A
:1022900089278783F0010BD08F91EF91FF9187837E
:1022A000089567D204D089C10F0101D089C100E02F
:1022B00077D209F008959A01281B390B1AF4D0013E
:1022C0000F01F5CF00272733300708F09CC2822F7B
:1022D000A7D1BBD1C9D1372F36270AF4EDD1F001F0
:1022E0008081A80E8181B81E8281C81E8381D81E7C
:1022F0008481E81E8581F81E86818F708061081FA9
:102300001AF4DAD180E8682705FF02C081E0AAD17B
:1023100004FD01C004D2C2C12CD204D04EC10F01B1
:1023200001D04EC108E13CD209F00895480F591F71
:102330004F5F534067276F935F934F9320D22227BD
:10234000F00179D193E0110F331F441F551F661F11
:10235000771F881F9A95B9F7FD01A7E0BB279191D8
:10236000A13011F49F709061992301F1939FA00C0B
:10237000B11CBB1F959FB695C01CD11CBB1F979F5E
:10238000B695E01CF11C0B1F919F200DA11CBB1FDB
:10239000949FB695B01CC11CBB1F969FB695D01CD0
:1023A000E11CBB1F989FB695F01C011DAA9549F032
:1023B0002A2DAB2CBC2CCD2CDE2CEF2CF02E0027A4
:1023C000CECF4F915F916F9104FB16F05ED102C0AA
:1023D0004F5F5F4F63C1FF9309901124F8E00694AB
:1023E00008F4190E17940794FA95D1F7FF91089500
:1023F000C0D104D0E2C00F0101D0E2C004E2D0D1CC
:1024000009F00895481B590B41505C4F67276F93A3
:102410005F934F93F00104D12FEFFD010CD1ADE399
:10242000BA2FB77019F420952F932FEFA116B3068A
:10243000C406D506E606F706080738F0A11AB30A5F
:10244000C40AD50AE60AF70A080B221FAA0CBB1C0D
:10245000CC1CDD1CEE1CFF1C001FAA9509F7209563
:10246000AF90BF90CF90DF90EF90FF900F914F9182
:102470005F916F9104FB1EF008D1415050400EC196
:10248000E881F981AA81BB810895FADF02D0FD01BC
:1024900082C0A1D0C5D0AC01632F61FD70C160FDC9
:1024A0006EC162FD77C14E5F534022F119F1552391
:1024B000A9F7463398F7483048F00F2DFE2CED2C45
:1024C000DC2CCB2CBA2CAA244850A8F7413048F079
:1024D000AA0CBB1CCC1CDD1CEE1CFF1C001F4150B9
:1024E000A9F7702F707E0F714EEF53E018D135D1E0
:1024F000A9F2FBC059C0E0EEF8E203C0E0EEF8E25A
:102500000DC05D01FF93EF9307D2EF91FF913CD097
:10251000F501FA93EA93C8DE22960CC25D01FF939F
:10252000EF93FAD1EF91FF912FD0F501FA93EA934F
:10253000A6DE2296FFC1A881B981661778E06FB741
:102540008D9195917A9599F06FBF89076FB7F8CF04
:10255000E881F981AA81BB81661778E06FB78D9118
:1025600091917A9521F06FBF89076FB7F8CF70E826
:10257000872797276FBF890731F06FB7892B12F034
:1025800071E067276FBF089588E005900D928A95E6
:10259000E1F718970895A082B182C282D382E482C3
:1025A000F582068317830895A080B180C280D3800E
:1025B000E480F580068117810895EC81FD81EBCFE1
:1025C000E881F981E8CF88E091919D938A95E1F7C0
:1025D00018973897089586819781332797FB37F9A5
:1025E00088949F7721F4882311F4326008952FEEA8
:1025F00028172FE7290740F42FE02823089411F427
:102600003160089534600895807F969587959695FA
:10261000879596958795969587959894889408952B
:10262000A080B180C280D380E480F58006810F70E5
:102630000061222708951081318142815381648194
:10264000758186818F7080610895883050F02A2DC1
:10265000AB2CBC2CCD2CDE2CEF2CF02E0027885080
:10266000F4CF0895689401C0E894882369F0059533
:10267000F794E794D794C794B794A794279516F442
:102680004F5F5F4F8A95F1CF0895220FAA1CBB1CA4
:10269000CC1CDD1CEE1CFF1C001F089501D025C0C2
:1026A000203848F011F4A0FE06C0089412D005FFAF
:1026B000089581E0D7CF08952095A094B094C09458
:1026C000D094E094F09400950F9200240894201D7B
:1026D0000F9050F40F920024A01CB01CC01CD01C02
:1026E000E01CF01C001D0F9008955523B2F0352F0B
:1026F000342B99F03FEF431737E0530778F4440F3A
:10270000551F440F551F440F551F440F551F0F7E73
:10271000042B152F67FB17F9089531C037C087E0E8
:102720003F2D303230E0030778F40F2DFE2CED2CD6
:10273000DC2CCB2CBA2CA22E2227485050408A9554
:1027400079F7442755271BC088E004FD05C09DDFAD
:10275000415050408A95C9F708950F9200240A28E5
:102760000B280C280D280E280F28002A00200F9077
:102770000895EA81FB81A881B9810F010895AA24F7
:10278000BB2465017501850198940895F8DF00EF79
:102790001FE708958FEFA82EB82EF3DF1F77089557
:1027A0001ADF632FAC01FD0116DF732F00C0372F36
:1027B000362B3F7709F4089532FDECCF262F2727DB
:1027C000372F60FB32F961FB33F93F70E8EEF8E236
:1027D000002311F427FD3C96030FE00F0027F01FA4
:1027E000849187FDD7CF86FDD1DF85FDC8DF84FDCD
:1027F0000AD083FD0AD082FD0AD081FD0BD080FD76
:102800000BD098940895F001CFCEFD01CDCE67FB9B
:1028100017F9089577FBFCCF27FBFACFCD90DD9019
:10282000ED90FD90AA24BB240027112722276627BC
:10283000FF2012F406D0606843E254E070DF55DFF9
:10284000AACEC094D094E094F09481E0C80E88277A
:10285000D81EE81EF81E0895BEDE31FD19C032FDF7
:1028600017C030FD2AC08E5F934092F0992329F55E
:10287000803238F4D5DE81958B5DE7DEE894F4DEB6
:102880000CC0CC24C094DC2CEC2CFC2CF69412C094
:10289000CC24DD24EE24FF2410C080E8B81650F0CC
:1028A00031F4BA28B22AB81611F4C0FC03C0CDDF47
:1028B000F7FCE7CF37FF01C0C4DFCD92DD92ED9288
:1028C000FD920895B7FE089590E8B91611F4D0FE70
:1028D00008959FEFD91AE90AF90A09F403950895B2
:1028E000000000000000F03F000810001010100071
:1028F00008082000000810001080100008082000C0
:102900000041200041418000208020000020440040
:10291000418044002020800088E00FB6F8945A924D
:102920004A92E42DF52DA42DB52D480E8827581E6A
:102930000FBE08950FB6F894499059900FBE0895B0
:102940005A924A92480E591E08955A924A92480E37
:102950008827581E0895480E8827581E08950F92FC
:102960001F922F92C801D901489F80014A9F900170
:102970004B9F202C499F100D211D321D5A9F202C4A
:10298000589F100D211D321D599F200D311D689F2C
:10299000200D311D699F300D789F300D2F901F90B5
:1029A0000F9008950E94C4150D920020D9F7089544
:1029B000903029F08C91880F9A95E9F78C930895BF
:1029C000903071F00D911D912D913C91000F111FD0
:1029D000221F331F9A95D1F73C932E931E930E938B
:1029E0000895903029F08C9186959A95E9F78C930B
:1029F0000895903071F00D911D912D913C91369577
:102A00002795179507959A95D1F73C932E931E938A
:102A10000E93089533D0992711278F2D880F80E8C2
:102A2000F82A802F881F08F41FEF41F08F57082FD6
:102A300007FD04C0003240F08FEF01C08827982FB7
:102A4000D82EE82EF82E09C08FE1801B082FF694AF
:102A5000E794D79497950A95D1F7112351F0909563
:102A6000D094E094F09481E0980F8827D81EE81E57
:102A7000F81E0F2DFE2CED2CD92E0895D190E1904B
:102A8000F19001910895102F90E8FF0C001F092785
:102A9000990FF7941078652F90E8440F551F592728
:102AA000990F4795607800380895FF0C90E89027BB
:102AB000110F9795F794092F0895102FBD2CDE2C38
:102AC000EF2CF02E11234AF4B094D094E094F094BB
:102AD0009FEFB91AD90AE90AF90A0EE1FF2039F481
:102AE000FE2CED2CDB2CBB240850C2F716C032F0B4
:102AF0000A95BB0CDD1CEE1CFF1CF9CF0E94621472
:102B0000D4CFDD92ED92FD920C9308959FE7092FAB
:102B1000F92A9FEFD92EE92E0895DD24EE24FF2413
:102B2000002711270895AFDFC1F35038B1F31627FE
:102B3000005850580894051F12F418F4E7CF08F015
:102B4000ECCF0BD0FF202AF0BB0CDD1CEE1CFF1CD1
:102B5000ACCF0F5F0BF4DACFA8CF9F929924AA24B1
:102B6000BB24992788E1990CAA1CBB1CDD1CEE1C18
:102B7000FF1C30F4920EA31EB41ED91EE91EF91ECE
:102B80008A9589F79F900895C895319600200895F9
:102B9000FBDF202DF9DF302DF7DF402DF5DF502D45
:102BA000089591E005C092E003C094E001C098E070
:102BB000EBDF0D929A95E1F70895E80FF91FF1CF39
:102BC0002E2E3F2E992781918D3209F093958823DF
:102BD000D1F79A95E22DF32D112361F0091718F022
:102BE00011F0101B01C0191B28F021F080E28D9319
:102BF0001A95E9F780818D3219F48D93319604C0CE
:102C0000222311F08BE28D93091738F031F0091B64
:102C100021F080E38D930A95E9F781918D938823C4
:102C2000E1F7332351F0EA2FFB2F319633958E9144
:102C300082933A95E1F78EE28C930895040F151F65
:102C4000261F371F0895041B150B260B370B0895FD
:102C500004171507260737070895000F111F221FB5
:102C6000331F089500951095209530950F5F1F4FE5
:102C70002F4F3F4F0895019110810EC00191119186
:102C8000219130810BC00191108117FF05C03FEFEA
:102C90002FEF04C0008111272227332737FF03C0FD
:102CA000E1DF8DE28D93CF93DF93CF92DF92EF92AE
:102CB000AA24BB24CC24DD24EE2440E2CAE0DD2794
:102CC00055E093E38881890F87FD9F7083FD907F96
:102CD000891B89935A95A9F7C0DFAA1CBB1CCC1C81
:102CE000DD1CEE1C4A9551F7E894EFE0FF27829136
:102CF0000ED0EB30E0F71EF068948A2D0CD08827B8
:102D00008D93EF90DF90CF90DF91CF910895982F22
:102D1000829501D0892F8F70805D26F0803309F471
:102D2000089568948D93089500271127222733274B
:102D30001DD08A3328F4803318F005D015D0F9CF90
:102D40000EF490CF089580538F93402F512F622F10
:102D5000732F83DF82DF72DF80DF8F919927080F67
:102D6000191F291F391F08958D910895E894FCDFDC
:102D70008032E9F38B32D9F38930C9F38D3211F403
:102D80006894F2CF089588278D93089581918D934B
:102D90008823E1F7089594E081918D939A95E1F766
:102DA000089509919191992351F08A95D9F7319716
:102DB00081918D930A9519F08823D1F70895E3CF77
:102DC000E199FECFEEBBFFBB3196089591E001C0C3
:102DD00092E07B3751F47FB7F894F2DF8D918DBB91
:102DE000E29AE19A9A95C9F77FBF7727089591E013
:102DF00001C092E0E5DFE09A8DB38D939A95D1F70B
:102E00000895FF93881BF9E0001FFA9511F4FF91D4
:102E10000895881F841B18F4840F8894F5CF0894B4
:102E2000F3CF8FEF83959D919923E1F708956894EF
:102E300001C0E894AF93BF938D9116F0919103C0B8
:102E40000E94C415902D891718F011F48823A1F75A
:102E5000BF91AF910895E89463F80895689463F87A
:102E60000895A998A898A198A0980895A09AA198C3
:102E700003D0A09801D0A19AEF93FF93EAE0F0E08D
:102E80000E942411FF91EF910895A09AA19AF4DF76
:102E9000A098989BFECFF0DFA198EECF0894111F69
:102EA00001C0110F69F0A09A18F40000A19802C0A7
:102EB000A19A00C0E1DFA098989BFECFDDDFF1CFA3
:102EC000A09AA198D9DFA098989BFECFE8949999F1
:102ED000689462F8D1CF089401C08894331F11E040
:102EE000A09AA198C9DFA098989BFECFC5DF8894CF
:102EF00099990894111FA0F7A09A379510F4A198FA
:102F000001C0A19AB9DFA098989BFECFB5DF0895C4
:102F10000000000000000000000000000000B041C0
:102F20000000000000DB8A410000001023459B41A7
:102F300000000010EE389B4100000020673F9B41DD
:102F400000000000000059404260653B49463B00DC
:102F5000494600003B00464100005A5A50413B00A0
:062F60005A5A5041000026
:00000001FF
